:020000040000FA
:100000008E018F0190019101023092000130930026
:1000100094018501860183168501803086000430B5
:1000200081008312861FCF28372072200B1D1628CF
:100030008B01A1200C08143A031D222830308600C1
:100040001F3085008C0B162814280F398207403486
:10005000793424343034193412340234783400348E
:1000600010347F347F347F347F347F347F347A3070
:100070008C008E0A0E08093C031808007B308C00A7
:100080008E018F0A0F08053C0318080079308C0098
:100090008F01900A1008093C031808007B308C007F
:1000A0009001910A1108053C031808007C308C006F
:1000B00091011308003C03186828920A1208023CB8
:1000C000031808007D308C009201920A9301080009
:1000D000920A1208093C031808007D308C00920136
:1000E000930A08009501940A1408083C031C940123
:1000F0001408013A03198A28033A03198F28013A90
:1001000003199228073A03199528303086001F30CA
:100110008500080095151308031D9728080015157C
:10012000120897289514110897281514100897009D
:1001300025208D001F3985000D0C303915048600EF
:100140000800861B0800950803190800970A17087D
:10015000093C031C970117089720C720861FAE286B
:10016000C720861FAE2814309600861FA628C720F9
:10017000960BB528170894018F018E0195199300ED
:1001800015199200951891001518900014280C303C
:100190008C000B1DC9288B018C0BC9280800960107
:1001A00016089720C720C720960A16080A3A031D8A
:0401B000D028CF285C
:02400E00F93F78
:00000001FF
